:020000040000FA
:02000000B52D1C
:08000800FF00030E8301FE005E
:100010008312031300308A0023308100A20A0530C6
:1000200022020318A2012114A30F1928A40F1928D2
:10003000A1145708003E03193828481C3628831697
:10004000031339308500831203138514C72201304E
:10005000D12200001E30A50085100730D122851462
:100060000630D122A50B2C2885105028C72239280C
:10007000BC222E30A6000830FD00220803195820AB
:100080000130220203197420023022020319902049
:10009000033022020319AC20043022020319C820C5
:1000A000373085000B117E0E8300FF0E7F0E090096
:1000B000E420A60B58286121E4206721E420752163
:1000C000E420C022E42085196D2810304502031871
:1000D0006B28C50A7328421573284508031972282E
:1000E000C503732842110800FD20A60B7428612166
:1000F000FD206721FD207521FD20C022FD208519EE
:1001000089281030460203188728C60A8F28C2158E
:100110008F28460803198E28C6038F28C2110800AD
:100120001621A60B90286121162167211621752121
:100130001621C02216218519A52810304702031860
:10014000A328C70AAB284216AB2847080319AA28D8
:10015000C703AB28421208004821A60BAC28612136
:1001600048216721482175214821C022482185194D
:10017000C128103043020318BF28C30AC7284214FD
:10018000C72843080319C628C303C728421008001C
:100190002F21A60BC82861212F2167212F2175212E
:1001A0002F21C0222F218519DD2810304402031889
:1001B000DB28C40AE328C214E32844080319E22810
:1001C000C403E328C210080001082B02031CFD141D
:1001D00001082F02031C7D1501083302031C7D1644
:1001E00001083702031CFD16831603137D088500E2
:1001F0008312031336308500080001082702031C10
:100200007D1401083002031C7D1501083402031C13
:100210007D1601083802031CFD16831603137D08A2
:100220008500831203133530850008000108280279
:10023000031C7D1401082C02031CFD140108350267
:10024000031C7D1601083902031CFD1683160313D7
:100250007D088500831203133330850008000108F0
:100260002902031C7D1401082D02031CFD14010842
:100270003102031C7D1501083A02031CFD1683168A
:1002800003137D08850083120313273085000800BF
:1002900001082A02031C7D1401082E02031CFD1410
:1002A00001083202031C7D1501083602031C7D166D
:1002B000831603137D08850083120313173085000E
:1002C000080003103B0DC9006E21CC00080003108C
:1002D0003B0D013EC9006E21CD00080001308A00AF
:1002E0004908793E03188A0A82004C088A004D08A2
:1002F00082000134B9340134C1340134C9340134C9
:10030000D1340134D9340134E1340134E9340134D5
:10031000F4340134F834023404340234083402343E
:1003200014340234183402342434023428340234AD
:10033000343402343834023444340234483402341D
:10034000543402345834023464340234683402348D
:1003500074340234783402348434023488340234FD
:100360009434023498340234A4340234A83402346D
:10037000B4343D18BE290630BB00B62A0130BB009C
:10038000B62A3D18C6290030BB00B62A0230BB0091
:10039000B62A3D18CE290030BB00B62A0330BB0078
:1003A000B62A3D18D6290430BB00B62A0330BB005C
:1003B000B62A3D18DE290030BB00B62A0530BB0046
:1003C000B62A3D18E6290730BB00B62A0030BB002C
:1003D000B62A3D18F22900304B070319F129CB0B3F
:1003E000B62AB62ABB01B62A3D08C100BB0AB62A06
:1003F00041083D06031DFE29BB01B62A3D184010E9
:100400003D1C4014BB0AB62A3D08C100BB0AB62AEF
:1004100041083D06031D0E2ABB01B62A3D183F12B6
:100420003D1C3F16BB0AB62A3D08C100BB0AB62ACE
:1004300041083D06031D1E2ABB01B62A3D18BF1107
:100440003D1CBF15BB0AB62A3D08C100BB0AB62A2F
:1004500041083D06031D2E2ABB01B62A3D183F1157
:100460003D1C3F15BB0AB62A3D08C100BB0AB62A8F
:1004700041083D06031D3E2ABB01B62A3D18BF10A8
:100480003D1CBF14BB0AB62A3D08C100BB0AB62AF0
:1004900041083D06031D4E2ABB01B62A3D183F10F8
:1004A0003D1C3F14BB0AB62A3D08C100BB0AB62A50
:1004B00041083D06031D5E2ABB01B62A3D18BE1247
:1004C0003D1CBE16BB0AB62A3D08C100BB0AB62AAF
:1004D00041083D06031D6E2ABB01B62A3D183E1297
:1004E0003D1C3E16BB0AB62A3D08C100BB0AB62A0F
:1004F00041083D06031D7E2ABB01B62A3D18BE11E8
:100500003D1CBE15BB0AB62A3D08C100BB0AB62A6F
:1005100041083D06031D8E2ABB01B62A3D183E1137
:100520003D1C3E15BB0AB62A3D08C100BB0AB62ACF
:1005300041083D06031D9E2ABB01B62A3D18BE1088
:100540003D1CBE14BB0AB62A3D08C100BB0AB62A30
:1005500041083D06031DAE2ABB01B62A3D183E10D8
:100560003D1C3E14BB0AB62ABB014A1408004210C7
:10057000C210851E421408003D1085193D14080064
:100580003C083B02031CC62A3B08BC00080048107C
:10059000D7030310D60CD50CD40CD30C0318481475
:1005A0000800CE00CE0BD22A0800D401D501D60116
:1005B000A030D300D109511C54145118D4144F1E2B
:1005C00054154F1AD415CF1D5416CF19D4164F1DDC
:1005D00054174F19D417CF1C5514CF18D5144F1CCE
:1005E00055154F18D515D01E5516D01AD516501EB4
:1005F0005517501AD517D01D5614D019D614501DA2
:1006000056155019D615D01C5616D018D616501C93
:1006100056175018D6172130D7000800D801D90135
:100620000830DA000310DC0CD90DD80DDB0CD90D25
:10063000D80DDA0B122B0800DD000000DD0B1D2B9E
:100640000800E50A65080F3C0319E5016508D200BA
:10065000FC010800E5036508013E031D322B0E3046
:10066000E500D200FC0108003E08E500D200F13EA2
:10067000031C3E2B0E30E5026508372BFC010800F9
:10068000DE002110211C422BDE0B412B0800650AE5
:10069000E700DC00DB010E235808E7005908E800FA
:1006A000E901E0306C18E900FF30C724E701E801F8
:1006B000E9010130C72408000630DF003730E000D0
:1006C0000310650DFC008B132A268B17E200031420
:1006D000650DFC008B132A268B17E0006208DF00F3
:1006E000080021305F02031D792B60087C07A223DC
:1006F0008B2B8B130A08E3005F087B07F3000310C2
:1007000060087C07F4000318F30A3126E40063084C
:100710008A0064088B17FC0F8E2BFB0A08008316D7
:1007200003139C18912B8B131C157C089B007A08D3
:100730009A0055309D00AA309D009C148B1783129F
:10074000031308008B13831603139C18A52B1C118D
:100750009B009C131C141A08831203138B170800A8
:100760009730A223EC000800B0236C1CB92B6C104E
:10077000BA2B6C149730FC006C08FA008F234723C7
:10078000472308005C23FC01FB017123E600E6130C
:100790007123EB00EB0A7123ED004A1CEB2B0730B1
:1007A0003F02031DD62B3423CA01C22BBF08031DF1
:1007B000EB2B20303E020319212321303E02031986
:1007C0002A2300303E020319E5010C303E020319D2
:1007D000B423CA01C22B42080319052C472347231F
:1007E000033042020319F32D0C3042020319B423E3
:1007F0004218FD2BC218012CC22B2123472347236B
:10080000F02B2A2347234723F02B063066020319D7
:100810002C241330660204308A0003193D2403306F
:100820008A001530660206308A0003195526033007
:100830008A005708003E031D292CA11C292CA11059
:100840006C1C242C2123C22B0730CF005208D0006F
:10085000D522ED0BCD2BC22B7123E7007123E800CD
:100860007123E9001F306905EE00EE0AEE0DEE0D72
:100870006B08C724EE0B382C08007123E7007123A6
:10088000E8000F306805EF000F306F02031D4D2C9C
:10089000E701E801E901C724BC2CE71B822C671F94
:1008A000682C3408BA002B08B4003908AB003508AE
:1008B000B9002F08B5003808AF003708B800330872
:1008C000B700B30140306718B307A030E718B3078B
:1008D000E71E812C2D08B6002708AD003208A700BE
:1008E0003108B2002808B1002E08A8002A08AE007E
:1008F0002908AA00A90140306719A907A030E71903
:10090000A907B42C671F9B2C3708B3003808B70021
:100910002F08B8003508AF003908B5002B08B9001A
:100920003408AB003A08B400BA0140306718BA077F
:10093000A030E718BA07E71EB42C2A08A9002E0831
:10094000AA002808AE003108A8003208B100270824
:10095000B2002D08A7003608AD00B6014030671977
:10096000B607A030E719B6076B0840234218BC2C25
:100970004A18BC2CEF0B4D2C0800700D700D701A2E
:10098000013AF01A013AF019013AF0000800EA00C1
:10099000B301E71BB309B701E71AB709B801E719B3
:1009A000B809AF01E718AF09B501E81BB509B901EE
:1009B000E81AB909AB01E819AB09B401E818B409A0
:1009C000BA01E91BBA09A901671BA909AA01671A9B
:1009D000AA09AE016719AE09A8016718A809B101F3
:1009E000681BB109B201681AB209A7016819A70901
:1009F000AD016818AD09B601691BB609AC01B001BB
:100A00006A084023080002303B02031C0301E70090
:100A10000030E8000130C724420803193D2DBC0115
:100A2000BB015708003E031D0C2D4208E800E701FA
:100A30000130C724CF01033042020319F32D4218BD
:100A4000292DC2182D2D4219312DC219352D421ACA
:100A5000392D2030D000D5220C2D2130D000D522C8
:100A60000C2D1030D000D5220C2D1130D000D52205
:100A70000C2D0C30D000D5220C2D4A1C032DCA01A0
:100A8000F030E700E8017F30C724E701E8013F309C
:100A9000C724F030E700E8017F30C7243E08E700B4
:100AA0003F08E800FF30C724FF30C724BC01BB016A
:100AB000032D9D25033042020319F32D42189D2575
:100AC0000130710203197A2D0230710203197F2D52
:100AD000033071020319842D0430710203198A2D29
:100AE000053071020319902D063071020319952DFE
:100AF0009D255A2DE701C030E800E9019A2D0C3000
:100B0000E700E800E9019A2D0C30E700CC30E8005E
:100B1000E9019A2DCC30E700E9000C30E8009A2D6D
:100B2000CC30E700E800E8009A2DCF30E700E9007C
:100B30003C30E800FF30C7245A2DE40ABD2455306C
:100B4000E700E800E900FF30C724AA30E700E8002A
:100B5000E900FF30C72442189D2D70082307640761
:100B6000F100F10C0730F105080085018101E50174
:100B7000D701C001BF01BE01C101BB01BC01CA0157
:100B8000A201A301A4010730990083160313823048
:100B9000810070308F049F0183120313C2011D3046
:100BA000F0008B168B17FF30E700E800E900FF30FC
:100BB000C724FF30C724FF30C724FF30C724E70114
:100BC000E801E901FF30C724FF30C724FF30C72404
:100BD000B0234208E800FF30C724FF30C724F201E9
:100BE00042080319C22BE701720ADC00DB010E2365
:100BF0005808E8005908E900E80CE90CE80CE90C91
:100C0000E80CE90CE80CE90CFF30C724FF30C724DE
:100C100042181C26C2182226421A0F2EF32D00302D
:100C200072020319C22B013072020319032D023024
:100C300072020319592DF32DF20A7208033C0319AD
:100C4000F2010800F2037208013E031D292E023052
:100C5000F20008005F088A007C08600703188A0A0F
:100C600082000A08E30073088A00740882000634D0
:100C7000DF340634FA340734093407341B340734BC
:100C8000303407344E34073457340734753407345E
:100C900084340734C9340734D03421340134213446
:100CA0003D342134493421348B3403308A0071239C
:100CB000E7007123E8007123E9003F306905EE0089
:100CC000EE0DEE0D29308400E71BD726E71FDB264B
:100CD0002A308400E71AD726E71EDB262E30840050
:100CE000E719D726E71DDB2628308400E718D7262A
:100CF000E71CDB2631308400E81BD726E81FDB2603
:100D000032308400E81AD726E81EDB26273084001C
:100D1000E819D726E81DDB262D308400E818D726F1
:100D2000E81CDB2636308400E91BD726E91FDB26CA
:100D300033308400671BD726671FDB2637308400DB
:100D4000671AD726671EDB26383084006719D72636
:100D5000671DDB262F3084006718D726671CDB262B
:100D600035308400681BD726681FDB2639308400A5
:100D7000681AD726681EDB262B3084006819D72610
:100D8000681DDB26343084006818D726681CDB26F3
:100D90003A308400691BD726691FDB266B08402385
:100DA0004218D62E4A18D62EEE0B622E0800800A64
:100DB0000319800908008008031D8003080013340C
:100DC00040340C34BF340134B0340934DF340134DE
:100DD000D0340934FF340134F03409343F34013461
:100DE000303409345F340134503409347F340134F1
:100DF0007034093406343034043440340034403420
:100E00001034013400340434043400340134103418
:100E10000034153410340534553455345F34AA3455
:100E2000AA349F34003400341F340034C0340F34EB
:100E3000FF34FF34DF34153403340634553455346D
:100E40007F34003400343F34AA34AA34BF34003431
:100E500000343F34FF34FF34FF34003400343F3477
:100E6000153403340934043400341F34043400349A
:100E70001F341C3410341F34783470345F34E13440
:100E8000E134DF34833487349F3402340E341F342A
:100E9000003408341F34003400343F340634303416
:100EA0000234553455344034AA34AA34A0340634BC
:100EB00030340934803400344034403400348034D9
:100EC0002034013400341034023400340834043443
:100ED0000034043408340034023410340034013453
:100EE000203400340034C034003406341034043468
:100EF0001134113400342234223420344434443444
:100F0000403488348834803406341734163411342D
:100F100011340034223422342034443444344034F4
:100F2000883488348034113411340034223422342B
:100F30002034443444344034883488348034113488
:100F400011340034223422342034443444344034C4
:100F50008834883480344434443440342234223455
:100F600020341134113400348834883480344434CB
:100F700044344034223422342034113411340034C7
:100F80008834883480344434443440342234223425
:100F90002034133440340234FC340934F33409343B
:100FA000133480340C34B53409343A340934BF3442
:100FB00009343A340934B5340934303409347534D9
:100FC0000934FA3409347F340934FA340934753475
:060FD0000934F03409347D
:02400E00C430BC
:10420000FF000600050013000034003420340034A1
:104210000034803400340234003400340834003474
:10422000003420340034003480340034023400344C
:104230000034083400340034203400340034803436
:10424000003400344034003400341034003400347E
:104250000434003400340134003400340034403479
:10426000003400341034003400340434003400349A
:1042700001340034003400344034060010000300E0
:1042800092344934203449342434803424349234F0
:10429000403406000500150000340034203400349A
:1042A00000348034003402340034003408340034E4
:1042B00000342034003400348034003402340034BC
:1042C00000340834003400342034003400348034A6
:1042D00000340034003400340034003400344034FE
:1042E0000034013400340034043400340034103419
:1042F00000340034403400340134003400340434D9
:1043000000340034103400340034403400340034BD
:1043100000340034003406001000030092344934A5
:1043200020342434923440344934243480340034EA
:00000001FF
